:020000021000EC
:10FC000001C020C1112484B7882391F00E98169A60
:10FC100090B1282F2A70223011F496FF09C081FF7D
:10FC200002C097EF94BF282E80E0F7D00C9400001C
:10FC300085E08093810082E08093C00088E180931A
:10FC4000C10086E08093C20080E18093C40080E020
:10FC5000E4D0239A86E020E33CEF91E030938500E6
:10FC60002093840096BBB09BFECF1B9AA895409131
:10FC7000C00047FD02C0815089F743E0B42EAA249A
:10FC8000A39451E1752EBDD0813471F4BAD0C82F40
:10FC9000CAD081E0C23821F088E0C13809F083E0A1
:10FCA000A9D080E1A7D0EFCF823419F484E1C3D08A
:10FCB000F8CF853411F485E0FACF853581F4A1D0F1
:10FCC000082F9FD0182F87FF07C08BB781608BBF8D
:10FCD000000F111FA8D0E5CF8BB78E7FF8CF8635E8
:10FCE00081F48FD08D3459F48CD0CBB78AD0C170C9
:10FCF000880F8C2B8BBF81E09ED080E0D1CF83E03A
:10FD0000FBCF843609F046C07CD0E82EF12CFE2CC7
:10FD1000EE2477D0E82A75D0682EE701C12CDD24C7
:10FD2000D39446018FEFC81AD80A6BD0F4018083B0
:10FD30002197B9F778D0F5E46F120DC0FE01F39565
:10FD4000EC16FD0609F4ADCF6081CE01800F911F46
:10FD500091D02196F3CFF801B7BEE89507B600FC25
:10FD6000FDCFFE01E00FF11FDE01B3958D919C9157
:10FD70000C01A7BEE89511242296EC16FD0689F722
:10FD800085E0F80187BFE89507B600FCFDCF77BE98
:10FD9000E89587CF8437F9F434D0C82FD0E0DC2F32
:10FDA000CC272FD0C82B2DD0D82E3DD07801F5E40C
:10FDB000DF120AC0C70156D01DD021978FEFE81A75
:10FDC000F80A2097B9F76DCFF70187917F0112D01C
:10FDD0002197D1F766CF853739F425D08EE10AD047
:10FDE00087E908D085E05CCF813509F073CF88E0E2
:10FDF00014D070CF9091C00095FFFCCF8093C600C7
:10FE000008958091C00087FFFCCF8091C00084FDE1
:10FE100001C0A8958091C6000895E0E6F0E098E161
:10FE2000908380830895EDDF803219F088E0F5DF5C
:10FE3000FFCF84E1DFCFCF93C82FE3DFC150E9F7D5
:10FE4000CF91F1CFFC010A0167BFE895112407B6F5
:10FE500000FCFDCF667029F0452B19F481E187BFC6
:10FE6000E8950895F999FECF92BD81BDF89A99273A
:10FE700080B50895262FF999FECF1FBA92BD81BD96
:10FE800020BD0FB6F894FA9AF99A0FBE019608951C
:10FE900056657273696F6E3D382E31004F5054496C
:10FEA000424F4F545F435553544F4D5645523D308A
:10FEB000004465766963653D61746D6567613132E3
:10FEC00038347000465F4350553D31363030303065
:10FED00030304C00424947424F4F543D310042754B
:10FEE000696C743A41707220313820323032313AC4
:10FEF00032323A30333A303000554152543D3000BE
:10FF0000424155445F524154453D313135323030E4
:10FF1000004C45443D4233004C45445F53544152EC
:0CFF2000545F464C41534845533D3300AC
:02FFFE000108F8
:040000031000FC00ED
:00000001FF
